
 Start         Length     Name                   Class
 0001:00401000 0000048C4H _TEXT                  CODE
 0002:00406000 0000044E4H _DATA                  DATA
 0003:0040A4E4 00000125CH _BSS                   BSS
 0004:00000000 00000009CH _TLS                   TLS


Detailed map of segments
 0001:00000000 0000014F C=CODE    S=_TEXT    G=(none)   M=C:\PROGRAM FILES\BORLAND\BCC55\LIB\C0X32.OBJ ACBP=A9
 0001:00000150 000000FE C=CODE    S=_TEXT    G=(none)   M=C:\PROGRAMS\IBM\SOM\SAMPLES\SOMK\C\TP\MAIN.OBJ ACBP=A9
 0001:00000250 0000004A C=CODE    S=_TEXT    G=(none)   M=C:\PROGRAMS\IBM\SOM\SAMPLES\SOMK\C\TP\HELPER.OBJ ACBP=A9
 0001:0000029C 00000319 C=CODE    S=_TEXT    G=(none)   M=C:\PROGRAMS\IBM\SOM\SAMPLES\SOMK\C\TP\BLEP.OBJ ACBP=A9
 0001:000005B8 000000E8 C=CODE    S=_TEXT    G=(none)   M=C:\PROGRAMS\IBM\SOM\SAMPLES\SOMK\C\TP\BT.OBJ ACBP=A9
 0001:000006A0 00000567 C=CODE    S=_TEXT    G=(none)   M=C:\PROGRAMS\IBM\SOM\SAMPLES\SOMK\C\TP\COLBLK.OBJ ACBP=A9
 0001:00000C08 00000665 C=CODE    S=_TEXT    G=(none)   M=C:\PROGRAMS\IBM\SOM\SAMPLES\SOMK\C\TP\EP.OBJ ACBP=A9
 0001:00001270 000003FE C=CODE    S=_TEXT    G=(none)   M=C:\PROGRAMS\IBM\SOM\SAMPLES\SOMK\C\TP\FM.OBJ ACBP=A9
 0001:00001670 0000016E C=CODE    S=_TEXT    G=(none)   M=C:\PROGRAMS\IBM\SOM\SAMPLES\SOMK\C\TP\FOOTER.OBJ ACBP=A9
 0001:000017E0 0000016E C=CODE    S=_TEXT    G=(none)   M=C:\PROGRAMS\IBM\SOM\SAMPLES\SOMK\C\TP\HEADER.OBJ ACBP=A9
 0001:00001950 00000164 C=CODE    S=_TEXT    G=(none)   M=C:\PROGRAMS\IBM\SOM\SAMPLES\SOMK\C\TP\IPEP.OBJ ACBP=A9
 0001:00001AB4 000003A0 C=CODE    S=_TEXT    G=(none)   M=C:\PROGRAMS\IBM\SOM\SAMPLES\SOMK\C\TP\LINK.OBJ ACBP=A9
 0001:00001E54 00000A05 C=CODE    S=_TEXT    G=(none)   M=C:\PROGRAMS\IBM\SOM\SAMPLES\SOMK\C\TP\LL.OBJ ACBP=A9
 0001:0000285C 00000508 C=CODE    S=_TEXT    G=(none)   M=C:\PROGRAMS\IBM\SOM\SAMPLES\SOMK\C\TP\PAGE.OBJ ACBP=A9
 0001:00002D64 00000217 C=CODE    S=_TEXT    G=(none)   M=C:\PROGRAMS\IBM\SOM\SAMPLES\SOMK\C\TP\SUEP.OBJ ACBP=A9
 0001:00002F7C 0000040E C=CODE    S=_TEXT    G=(none)   M=C:\PROGRAMS\IBM\SOM\SAMPLES\SOMK\C\TP\TEXTLINE.OBJ ACBP=A9
 0001:0000338C 00000268 C=CODE    S=_TEXT    G=(none)   M=C:\PROGRAMS\IBM\SOM\SAMPLES\SOMK\C\TP\TPWORD.OBJ ACBP=A9
 0001:000035F4 00000B9A C=CODE    S=_TEXT    G=(none)   M=C:\PROGRAMS\IBM\SOM\SAMPLES\SOMK\C\TP\TXTEP.OBJ ACBP=A9
 0001:00004190 00000527 C=CODE    S=_TEXT    G=(none)   M=C:\PROGRAMS\IBM\SOM\SAMPLES\SOMK\C\TP\WORD.OBJ ACBP=A9
 0001:000046B8 00000001 C=CODE    S=_TEXT    G=(none)   M=C:\PROGRAM FILES\BORLAND\BCC55\LIB\CW32MTI.LIB|crtlst_i ACBP=A9
 0001:000046BC 00000001 C=CODE    S=_TEXT    G=(none)   M=C:\PROGRAM FILES\BORLAND\BCC55\LIB\CW32MTI.LIB|crtlst_l ACBP=A9
 0001:000046C0 0000009F C=CODE    S=_TEXT    G=(none)   M=C:\PROGRAM FILES\BORLAND\BCC55\LIB\CW32MTI.LIB|xxv ACBP=A9
 0001:00004760 00000026 C=CODE    S=_TEXT    G=(none)   M=C:\PROGRAM FILES\BORLAND\BCC55\LIB\CW32MTI.LIB|setargv2 ACBP=A9
 0002:00000018 000000A4 C=DATA    S=_DATA    G=DGROUP   M=C:\PROGRAM FILES\BORLAND\BCC55\LIB\C0X32.OBJ ACBP=A9
 0002:000000BC 00000074 C=DATA    S=_DATA    G=DGROUP   M=C:\PROGRAMS\IBM\SOM\SAMPLES\SOMK\C\TP\MAIN.OBJ ACBP=A9
 0002:00000130 000000C8 C=DATA    S=_DATA    G=DGROUP   M=C:\PROGRAMS\IBM\SOM\SAMPLES\SOMK\C\TP\HELPER.OBJ ACBP=A9
 0002:000001F8 000002FC C=DATA    S=_DATA    G=DGROUP   M=C:\PROGRAMS\IBM\SOM\SAMPLES\SOMK\C\TP\BLEP.OBJ ACBP=A9
 0002:000004F4 0000027C C=DATA    S=_DATA    G=DGROUP   M=C:\PROGRAMS\IBM\SOM\SAMPLES\SOMK\C\TP\BT.OBJ ACBP=A9
 0002:00000770 000003F0 C=DATA    S=_DATA    G=DGROUP   M=C:\PROGRAMS\IBM\SOM\SAMPLES\SOMK\C\TP\COLBLK.OBJ ACBP=A9
 0002:00000B60 0000075C C=DATA    S=_DATA    G=DGROUP   M=C:\PROGRAMS\IBM\SOM\SAMPLES\SOMK\C\TP\EP.OBJ ACBP=A9
 0002:000012BC 00000474 C=DATA    S=_DATA    G=DGROUP   M=C:\PROGRAMS\IBM\SOM\SAMPLES\SOMK\C\TP\FM.OBJ ACBP=A9
 0002:00001730 00000244 C=DATA    S=_DATA    G=DGROUP   M=C:\PROGRAMS\IBM\SOM\SAMPLES\SOMK\C\TP\FOOTER.OBJ ACBP=A9
 0002:00001974 00000244 C=DATA    S=_DATA    G=DGROUP   M=C:\PROGRAMS\IBM\SOM\SAMPLES\SOMK\C\TP\HEADER.OBJ ACBP=A9
 0002:00001BB8 00000280 C=DATA    S=_DATA    G=DGROUP   M=C:\PROGRAMS\IBM\SOM\SAMPLES\SOMK\C\TP\IPEP.OBJ ACBP=A9
 0002:00001E38 000004B4 C=DATA    S=_DATA    G=DGROUP   M=C:\PROGRAMS\IBM\SOM\SAMPLES\SOMK\C\TP\LINK.OBJ ACBP=A9
 0002:000022EC 00000794 C=DATA    S=_DATA    G=DGROUP   M=C:\PROGRAMS\IBM\SOM\SAMPLES\SOMK\C\TP\LL.OBJ ACBP=A9
 0002:00002A80 00000548 C=DATA    S=_DATA    G=DGROUP   M=C:\PROGRAMS\IBM\SOM\SAMPLES\SOMK\C\TP\PAGE.OBJ ACBP=A9
 0002:00002FC8 000002A8 C=DATA    S=_DATA    G=DGROUP   M=C:\PROGRAMS\IBM\SOM\SAMPLES\SOMK\C\TP\SUEP.OBJ ACBP=A9
 0002:00003270 000003CC C=DATA    S=_DATA    G=DGROUP   M=C:\PROGRAMS\IBM\SOM\SAMPLES\SOMK\C\TP\TEXTLINE.OBJ ACBP=A9
 0002:0000363C 00000228 C=DATA    S=_DATA    G=DGROUP   M=C:\PROGRAMS\IBM\SOM\SAMPLES\SOMK\C\TP\TPWORD.OBJ ACBP=A9
 0002:00003864 00000700 C=DATA    S=_DATA    G=DGROUP   M=C:\PROGRAMS\IBM\SOM\SAMPLES\SOMK\C\TP\TXTEP.OBJ ACBP=A9
 0002:00003F64 00000474 C=DATA    S=_DATA    G=DGROUP   M=C:\PROGRAMS\IBM\SOM\SAMPLES\SOMK\C\TP\WORD.OBJ ACBP=A9
 0002:000043D8 000000C4 C=DATA    S=_DATA    G=DGROUP   M=C:\PROGRAM FILES\BORLAND\BCC55\LIB\CW32MTI.LIB|xxv ACBP=A9
 0002:00004488 00000004 C=DATA    S=_DATA    G=DGROUP   M=C:\PROGRAM FILES\BORLAND\BCC55\LIB\CW32MTI.LIB|fmode ACBP=A9
 0002:0000448C 00000004 C=DATA    S=_DATA    G=DGROUP   M=C:\PROGRAM FILES\BORLAND\BCC55\LIB\CW32MTI.LIB|cfinfo ACBP=A9
 0002:00004490 00000004 C=DATA    S=_DATA    G=DGROUP   M=C:\PROGRAM FILES\BORLAND\BCC55\LIB\CW32MTI.LIB|xinitcvt ACBP=A9
 0002:00004494 00000004 C=DATA    S=_DATA    G=DGROUP   M=C:\PROGRAM FILES\BORLAND\BCC55\LIB\CW32MTI.LIB|setargv2 ACBP=A9
 0002:00004498 00000004 C=DATA    S=_DATA    G=DGROUP   M=C:\PROGRAM FILES\BORLAND\BCC55\LIB\CW32MTI.LIB|wildptr ACBP=A9
 0002:0000449C 00000004 C=DATA    S=_DATA    G=DGROUP   M=C:\PROGRAM FILES\BORLAND\BCC55\LIB\CW32MTI.LIB|wwildptr ACBP=A9
 0002:000044A0 00000004 C=DATA    S=_DATA    G=DGROUP   M=C:\PROGRAM FILES\BORLAND\BCC55\LIB\CW32MTI.LIB|xsetenvp ACBP=A9
 0002:000044A4 00000040 C=DATA    S=_DATA    G=DGROUP   M=<internal> ACBP=A9
 0003:00000000 00000028 C=BSS     S=_BSS     G=DGROUP   M=C:\PROGRAMS\IBM\SOM\SAMPLES\SOMK\C\TP\BLEP.OBJ ACBP=A9
 0003:00000028 00000010 C=BSS     S=_BSS     G=DGROUP   M=C:\PROGRAMS\IBM\SOM\SAMPLES\SOMK\C\TP\BT.OBJ ACBP=A9
 0003:00000038 00000030 C=BSS     S=_BSS     G=DGROUP   M=C:\PROGRAMS\IBM\SOM\SAMPLES\SOMK\C\TP\COLBLK.OBJ ACBP=A9
 0003:00000068 00000044 C=BSS     S=_BSS     G=DGROUP   M=C:\PROGRAMS\IBM\SOM\SAMPLES\SOMK\C\TP\EP.OBJ ACBP=A9
 0003:000000AC 00000028 C=BSS     S=_BSS     G=DGROUP   M=C:\PROGRAMS\IBM\SOM\SAMPLES\SOMK\C\TP\FM.OBJ ACBP=A9
 0003:000000D4 00000010 C=BSS     S=_BSS     G=DGROUP   M=C:\PROGRAMS\IBM\SOM\SAMPLES\SOMK\C\TP\FOOTER.OBJ ACBP=A9
 0003:000000E4 00000010 C=BSS     S=_BSS     G=DGROUP   M=C:\PROGRAMS\IBM\SOM\SAMPLES\SOMK\C\TP\HEADER.OBJ ACBP=A9
 0003:000000F4 00000018 C=BSS     S=_BSS     G=DGROUP   M=C:\PROGRAMS\IBM\SOM\SAMPLES\SOMK\C\TP\IPEP.OBJ ACBP=A9
 0003:0000010C 00000030 C=BSS     S=_BSS     G=DGROUP   M=C:\PROGRAMS\IBM\SOM\SAMPLES\SOMK\C\TP\LINK.OBJ ACBP=A9
 0003:0000013C 00000058 C=BSS     S=_BSS     G=DGROUP   M=C:\PROGRAMS\IBM\SOM\SAMPLES\SOMK\C\TP\LL.OBJ ACBP=A9
 0003:00000194 00000030 C=BSS     S=_BSS     G=DGROUP   M=C:\PROGRAMS\IBM\SOM\SAMPLES\SOMK\C\TP\PAGE.OBJ ACBP=A9
 0003:000001C4 00000010 C=BSS     S=_BSS     G=DGROUP   M=C:\PROGRAMS\IBM\SOM\SAMPLES\SOMK\C\TP\SUEP.OBJ ACBP=A9
 0003:000001D4 00000034 C=BSS     S=_BSS     G=DGROUP   M=C:\PROGRAMS\IBM\SOM\SAMPLES\SOMK\C\TP\TEXTLINE.OBJ ACBP=A9
 0003:00000208 0000000C C=BSS     S=_BSS     G=DGROUP   M=C:\PROGRAMS\IBM\SOM\SAMPLES\SOMK\C\TP\TPWORD.OBJ ACBP=A9
 0003:00000214 00000064 C=BSS     S=_BSS     G=DGROUP   M=C:\PROGRAMS\IBM\SOM\SAMPLES\SOMK\C\TP\TXTEP.OBJ ACBP=A9
 0003:00000278 00000FD4 C=BSS     S=_BSS     G=DGROUP   M=C:\PROGRAMS\IBM\SOM\SAMPLES\SOMK\C\TP\WORD.OBJ ACBP=A9
 0003:0000124C 00000008 C=BSS     S=_BSS     G=DGROUP   M=C:\PROGRAM FILES\BORLAND\BCC55\LIB\CW32MTI.LIB|xxv ACBP=A9
 0003:00001254 00000008 C=BSS     S=_BSS     G=DGROUP   M=C:\PROGRAM FILES\BORLAND\BCC55\LIB\CW32MTI.LIB|setargv2 ACBP=A9
 0004:00000000 0000009C C=TLS     S=_TLS     G=DGROUP   M=C:\PROGRAM FILES\BORLAND\BCC55\LIB\CW32MTI.LIB|xxv ACBP=A9

  Address         Publics by Name

 0001:00000140      Sysinit::__linkproc__ __fastcall GetTls()
 0001:00003393      TPWordNewClass
 0002:00003648      _TPWordCClassData
 0002:00003640      _TPWordClassData
 0002:000036B8      _TPWord_ClassInitBlock
 0003:0000124C      __DestructorCountPtr
 0001:000046EC      __ExceptInit
 0002:00004474      __ExceptVarsSize
 0001:00000059      __GetExceptDLLinfo
 0001:00004738      __GetExceptDLLinfoInternal
 0002:000000B4      __PackageInfoTable
 0002:000000A3      __TLS_index
 0002:000000A7      __TLS_index4
 0002:000000B0      ___CPPdebugHook
 0002:000000B0      ___CPPdebugHook_segment
 0002:000043D8      ___CPPexceptionList
 0001:000046BC      ___CRTL_VCLLIB_Linkage
 0001:000046B8      ___CRTL_VCL_Init
 0002:000043F4      ___ExceptStaticXbuff
 0001:00000140      ___System__GetTls
 0003:00001254      ___dll_argc
 0003:00001258      ___dll_argv
 0002:000043DC      ___exceptFlags
 0002:000043F0      ___exceptMemAllocVars
 0002:000043EC      ___exceptStaticBuffP
 0002:00000095      ___isDLL
 0002:0000005C      ___isGUI
 0002:00000094      ___isVCLPackage
 0002:000037B8      ___somC_TPWord_ClassInfo
 0002:00003674      ___somC_TPWord_newNDMethodsArray
 0003:00000208      ___somC_TPWord_parentMtabs
 0002:000006D4      ___somC_baseType_ClassInfo
 0002:00000568      ___somC_baseType_newNDMethodsArray
 0003:00000028      ___somC_baseType_parentMtabs
 0002:000003FC      ___somC_bulletedList_ClassInfo
 0003:00000020      ___somC_bulletedList_parentMtabs
 0002:00000A74      ___somC_columnBlock_ClassInfo
 0002:00000868      ___somC_columnBlock_newNDMethodsArray
 0003:00000050      ___somC_columnBlock_parentMtabs
 0002:000010F4      ___somC_envProcessor_ClassInfo
 0002:00000DA0      ___somC_envProcessor_newNDMethodsArray
 0003:00000070      ___somC_envProcessor_parentMtabs
 0002:00001628      ___somC_fileMgr_ClassInfo
 0002:000013EC      ___somC_fileMgr_newNDMethodsArray
 0003:000000B4      ___somC_fileMgr_parentMtabs
 0002:000018A8      ___somC_footer_ClassInfo
 0003:000000DC      ___somC_footer_parentMtabs
 0002:00001AEC      ___somC_header_ClassInfo
 0003:000000EC      ___somC_header_parentMtabs
 0002:00001D6C      ___somC_indentedParagraphs_ClassInfo
 0003:00000104      ___somC_indentedParagraphs_parentMtabs
 0002:000021A4      ___somC_link_ClassInfo
 0002:00001F68      ___somC_link_newNDMethodsArray
 0003:0000011C      ___somC_link_parentMtabs
 0002:000028C8      ___somC_linkedList_ClassInfo
 0002:000024EC      ___somC_linkedList_newNDMethodsArray
 0003:0000014C      ___somC_linkedList_parentMtabs
 0002:00002E98      ___somC_page_ClassInfo
 0002:00002C0C      ___somC_page_newNDMethodsArray
 0003:0000019C      ___somC_page_parentMtabs
 0002:000031A0      ___somC_setUpEnvProcessor_ClassInfo
 0002:00003034      ___somC_setUpEnvProcessor_newNDMethodsArray
 0003:000001C4      ___somC_setUpEnvProcessor_parentMtabs
 0002:00003540      ___somC_textLine_ClassInfo
 0002:0000334C      ___somC_textLine_newNDMethodsArray
 0003:000001F4      ___somC_textLine_parentMtabs
 0002:00003D80      ___somC_txtEnvProcessor_ClassInfo
 0002:00003A6C      ___somC_txtEnvProcessor_newNDMethodsArray
 0003:0000024C      ___somC_txtEnvProcessor_parentMtabs
 0002:000042B8      ___somC_word_ClassInfo
 0002:00004084      ___somC_word_newNDMethodsArray
 0003:00000290      ___somC_word_parentMtabs
 0002:000043E8      ___throwExceptionName
 0002:000043E0      ___throwFileName
 0002:000043E4      ___throwLineNumber
 0002:000000A2      ___useDynamicTLS
 0004:00000000      ___xxInfo
 0001:00000000      __acrtused
 0002:00004498      __argv_expand_ptr
 0002:0000448C      __fileinfo
 0002:00004488      __fmode
 0001:00000066      __getHInstance
 0002:000000AB      __hInstance
 0002:000044C4      __indStub:122
 0002:000044E0      __indStub:25
 0002:000044D8      __indStub:26
 0002:000044C0      __indStub:27
 0002:000044DC      __indStub:28
 0002:000044AC      __indStub:34
 0002:000044A4      __indStub:44
 0002:000044D4      __indStub:55
 0002:000044CC      __indStub:57
 0002:000044B0      __indStub:6
 0002:000044B8      __indStub:68
 0002:000044B4      __indStub:69
 0002:000044C8      __indStub:7
 0002:000044BC      __indStub:70
 0002:000044A8      __indStub:8
 0002:000044D0      __indStub:9
 0001:0000005E      __isDLL
 0002:00004494      __setargv__
 0002:000044A0      __setenvp__
 0002:00004490      __turboFloat
 0002:0000449C      __wargv_expand_ptr
 0002:00000504      _baseTypeCClassData
 0002:000004F8      _baseTypeClassData
 0002:000005D4      _baseType_ClassInitBlock
 0002:00000200      _bulletedListCClassData
 0002:000001FC      _bulletedListClassData
 0002:000002FC      _bulletedList_ClassInitBlock
 0002:00000788      _columnBlockCClassData
 0002:00000774      _columnBlockClassData
 0002:00000974      _columnBlock_ClassInitBlock
 0002:00000B9C      _envProcessorCClassData
 0002:00000B64      _envProcessorClassData
 0002:00000FF4      _envProcessor_ClassInitBlock
 0002:000012DC      _fileMgrCClassData
 0002:000012C0      _fileMgrClassData
 0002:00001528      _fileMgr_ClassInitBlock
 0002:00001738      _footerCClassData
 0002:00001734      _footerClassData
 0002:000017A8      _footer_ClassInitBlock
 0002:0000197C      _headerCClassData
 0002:00001978      _headerClassData
 0002:000019EC      _header_ClassInitBlock
 0002:00001BC0      _indentedParagraphsCClassData
 0002:00001BBC      _indentedParagraphsClassData
 0002:00001C6C      _indentedParagraphs_ClassInitBlock
 0002:00001E58      _linkCClassData
 0002:00001E3C      _linkClassData
 0002:000020A4      _link_ClassInitBlock
 0002:00002334      _linkedListCClassData
 0002:000022F0      _linkedListClassData
 0002:000027C8      _linkedList_ClassInitBlock
 0001:00000150      _main
 0002:00002AA8      _pageCClassData
 0002:00002A84      _pageClassData
 0002:00002D98      _page_ClassInitBlock
 0001:000034BB      _readToken
 0002:00002FD8      _setUpEnvProcessorCClassData
 0002:00002FCC      _setUpEnvProcessorClassData
 0002:000030A0      _setUpEnvProcessor_ClassInitBlock
 0001:00000250      _shouldHaveOverridden
 0001:000045DE      _showWordStats
 0002:00003284      _textLineCClassData
 0002:00003274      _textLineClassData
 0002:00003440      _textLine_ClassInitBlock
 0002:00003890      _txtEnvProcessorCClassData
 0002:00003868      _txtEnvProcessorClassData
 0002:00003C80      _txtEnvProcessor_ClassInitBlock
 0002:00003F80      _wordCClassData
 0002:00003F68      _wordClassData
 0002:000041B8      _word_ClassInitBlock
 0003:000000F4      b10_2
 0003:0000010C      b11_2
 0003:0000013C      b12_2
 0003:00000194      b13_2
 0003:000001C4      b14_2
 0003:000001D4      b15_2
 0003:00000208      b16_2
 0003:00000214      b17_2
 0003:00000278      b18_2
 0003:00000000      b3_2
 0003:00000028      b4_2
 0003:0000124C      b56_2
 0003:00000038      b5_2
 0003:00000068      b6_2
 0003:00001254      b78_2
 0003:000000AC      b7_2
 0003:000000D4      b8_2
 0003:000000E4      b9_2
 0001:000005BF      baseTypeNewClass
 0001:00000399      bulletedListNewClass
 0001:00001950      c10_0
 0001:00001AB4      c11_0
 0001:00001E54      c12_0
 0001:0000285C      c13_0
 0001:00002D64      c14_0
 0001:00002F7C      c15_0
 0001:0000338C      c16_0
 0001:000035F4      c17_0
 0001:00004190      c18_0
 0001:00000000      c19_0
 0001:00000150      c1_0
 0001:00000250      c2_0
 0001:0000029C      c3_0
 0001:000046B8      c40_0
 0001:000046BC      c44_0
 0001:000005B8      c4_0
 0001:000046C0      c56_0
 0001:000046C0      c56_4
 0001:000006A0      c5_0
 0001:00000C08      c6_0
 0001:00004760      c78_0
 0001:00004760      c78_3
 0001:00004780      c78_4
 0001:00001270      c7_0
 0001:00001670      c8_0
 0001:000017E0      c9_0
 0001:0000077B      columnBlockNewClass
 0002:00001BB8      d10_1
 0002:00001E38      d11_1
 0002:000022EC      d12_1
 0002:00002A80      d13_1
 0002:00002FC8      d14_1
 0002:00003270      d15_1
 0002:0000363C      d16_1
 0002:00003864      d17_1
 0002:00003F64      d18_1
 0002:00000018      d19_1
 0002:000000BC      d1_1
 0002:00000130      d2_1
 0002:000001F8      d3_1
 0002:000004F4      d4_1
 0002:000043D8      d56_1
 0002:00000770      d5_1
 0002:00004488      d62_0
 0002:0000448C      d64_0
 0002:00000B60      d6_1
 0002:00004490      d72_0
 0002:00004494      d78_1
 0002:000012BC      d7_1
 0002:00004498      d80_0
 0002:0000449C      d82_0
 0002:000044A0      d86_0
 0002:00001730      d8_1
 0002:00001974      d9_1
 0001:00000CB2      envProcessorNewClass
 0001:000012B7      fileMgrNewClass
 0001:000016B4      footerNewClass
 0001:00001824      headerNewClass
 0001:000019D2      indentedParagraphsNewClass
 0001:00001B3C      linkNewClass
 0001:00001EDC      linkedListNewClass
 0001:000028A3      pageNewClass
 0001:00002D6B      setUpEnvProcessorNewClass
 0004:00000000      t56_3
 0001:00003085      textLineNewClass
 0001:0000379B      txtEnvProcessorNewClass
 0001:0000426B      wordNewClass

  Address         Publics by Value

 0001:00000000      __acrtused
 0001:00000000      c19_0
 0001:00000059      __GetExceptDLLinfo
 0001:0000005E      __isDLL
 0001:00000066      __getHInstance
 0001:00000140      ___System__GetTls
 0001:00000140      Sysinit::__linkproc__ __fastcall GetTls()
 0001:00000150      c1_0
 0001:00000150      _main
 0001:00000250      _shouldHaveOverridden
 0001:00000250      c2_0
 0001:0000029C      c3_0
 0001:00000399      bulletedListNewClass
 0001:000005B8      c4_0
 0001:000005BF      baseTypeNewClass
 0001:000006A0      c5_0
 0001:0000077B      columnBlockNewClass
 0001:00000C08      c6_0
 0001:00000CB2      envProcessorNewClass
 0001:00001270      c7_0
 0001:000012B7      fileMgrNewClass
 0001:00001670      c8_0
 0001:000016B4      footerNewClass
 0001:000017E0      c9_0
 0001:00001824      headerNewClass
 0001:00001950      c10_0
 0001:000019D2      indentedParagraphsNewClass
 0001:00001AB4      c11_0
 0001:00001B3C      linkNewClass
 0001:00001E54      c12_0
 0001:00001EDC      linkedListNewClass
 0001:0000285C      c13_0
 0001:000028A3      pageNewClass
 0001:00002D64      c14_0
 0001:00002D6B      setUpEnvProcessorNewClass
 0001:00002F7C      c15_0
 0001:00003085      textLineNewClass
 0001:0000338C      c16_0
 0001:00003393      TPWordNewClass
 0001:000034BB      _readToken
 0001:000035F4      c17_0
 0001:0000379B      txtEnvProcessorNewClass
 0001:00004190      c18_0
 0001:0000426B      wordNewClass
 0001:000045DE      _showWordStats
 0001:000046B8      c40_0
 0001:000046B8      ___CRTL_VCL_Init
 0001:000046BC      c44_0
 0001:000046BC      ___CRTL_VCLLIB_Linkage
 0001:000046C0      c56_4
 0001:000046C0      c56_0
 0001:000046EC      __ExceptInit
 0001:00004738      __GetExceptDLLinfoInternal
 0001:00004760      c78_0
 0001:00004760      c78_3
 0001:00004780      c78_4
 0002:00000018      d19_1
 0002:0000005C      ___isGUI
 0002:00000094      ___isVCLPackage
 0002:00000095      ___isDLL
 0002:000000A2      ___useDynamicTLS
 0002:000000A3      __TLS_index
 0002:000000A7      __TLS_index4
 0002:000000AB      __hInstance
 0002:000000B0      ___CPPdebugHook_segment
 0002:000000B0      ___CPPdebugHook
 0002:000000B4      __PackageInfoTable
 0002:000000BC      d1_1
 0002:00000130      d2_1
 0002:000001F8      d3_1
 0002:000001FC      _bulletedListClassData
 0002:00000200      _bulletedListCClassData
 0002:000002FC      _bulletedList_ClassInitBlock
 0002:000003FC      ___somC_bulletedList_ClassInfo
 0002:000004F4      d4_1
 0002:000004F8      _baseTypeClassData
 0002:00000504      _baseTypeCClassData
 0002:00000568      ___somC_baseType_newNDMethodsArray
 0002:000005D4      _baseType_ClassInitBlock
 0002:000006D4      ___somC_baseType_ClassInfo
 0002:00000770      d5_1
 0002:00000774      _columnBlockClassData
 0002:00000788      _columnBlockCClassData
 0002:00000868      ___somC_columnBlock_newNDMethodsArray
 0002:00000974      _columnBlock_ClassInitBlock
 0002:00000A74      ___somC_columnBlock_ClassInfo
 0002:00000B60      d6_1
 0002:00000B64      _envProcessorClassData
 0002:00000B9C      _envProcessorCClassData
 0002:00000DA0      ___somC_envProcessor_newNDMethodsArray
 0002:00000FF4      _envProcessor_ClassInitBlock
 0002:000010F4      ___somC_envProcessor_ClassInfo
 0002:000012BC      d7_1
 0002:000012C0      _fileMgrClassData
 0002:000012DC      _fileMgrCClassData
 0002:000013EC      ___somC_fileMgr_newNDMethodsArray
 0002:00001528      _fileMgr_ClassInitBlock
 0002:00001628      ___somC_fileMgr_ClassInfo
 0002:00001730      d8_1
 0002:00001734      _footerClassData
 0002:00001738      _footerCClassData
 0002:000017A8      _footer_ClassInitBlock
 0002:000018A8      ___somC_footer_ClassInfo
 0002:00001974      d9_1
 0002:00001978      _headerClassData
 0002:0000197C      _headerCClassData
 0002:000019EC      _header_ClassInitBlock
 0002:00001AEC      ___somC_header_ClassInfo
 0002:00001BB8      d10_1
 0002:00001BBC      _indentedParagraphsClassData
 0002:00001BC0      _indentedParagraphsCClassData
 0002:00001C6C      _indentedParagraphs_ClassInitBlock
 0002:00001D6C      ___somC_indentedParagraphs_ClassInfo
 0002:00001E38      d11_1
 0002:00001E3C      _linkClassData
 0002:00001E58      _linkCClassData
 0002:00001F68      ___somC_link_newNDMethodsArray
 0002:000020A4      _link_ClassInitBlock
 0002:000021A4      ___somC_link_ClassInfo
 0002:000022EC      d12_1
 0002:000022F0      _linkedListClassData
 0002:00002334      _linkedListCClassData
 0002:000024EC      ___somC_linkedList_newNDMethodsArray
 0002:000027C8      _linkedList_ClassInitBlock
 0002:000028C8      ___somC_linkedList_ClassInfo
 0002:00002A80      d13_1
 0002:00002A84      _pageClassData
 0002:00002AA8      _pageCClassData
 0002:00002C0C      ___somC_page_newNDMethodsArray
 0002:00002D98      _page_ClassInitBlock
 0002:00002E98      ___somC_page_ClassInfo
 0002:00002FC8      d14_1
 0002:00002FCC      _setUpEnvProcessorClassData
 0002:00002FD8      _setUpEnvProcessorCClassData
 0002:00003034      ___somC_setUpEnvProcessor_newNDMethodsArray
 0002:000030A0      _setUpEnvProcessor_ClassInitBlock
 0002:000031A0      ___somC_setUpEnvProcessor_ClassInfo
 0002:00003270      d15_1
 0002:00003274      _textLineClassData
 0002:00003284      _textLineCClassData
 0002:0000334C      ___somC_textLine_newNDMethodsArray
 0002:00003440      _textLine_ClassInitBlock
 0002:00003540      ___somC_textLine_ClassInfo
 0002:0000363C      d16_1
 0002:00003640      _TPWordClassData
 0002:00003648      _TPWordCClassData
 0002:00003674      ___somC_TPWord_newNDMethodsArray
 0002:000036B8      _TPWord_ClassInitBlock
 0002:000037B8      ___somC_TPWord_ClassInfo
 0002:00003864      d17_1
 0002:00003868      _txtEnvProcessorClassData
 0002:00003890      _txtEnvProcessorCClassData
 0002:00003A6C      ___somC_txtEnvProcessor_newNDMethodsArray
 0002:00003C80      _txtEnvProcessor_ClassInitBlock
 0002:00003D80      ___somC_txtEnvProcessor_ClassInfo
 0002:00003F64      d18_1
 0002:00003F68      _wordClassData
 0002:00003F80      _wordCClassData
 0002:00004084      ___somC_word_newNDMethodsArray
 0002:000041B8      _word_ClassInitBlock
 0002:000042B8      ___somC_word_ClassInfo
 0002:000043D8      d56_1
 0002:000043D8      ___CPPexceptionList
 0002:000043DC      ___exceptFlags
 0002:000043E0      ___throwFileName
 0002:000043E4      ___throwLineNumber
 0002:000043E8      ___throwExceptionName
 0002:000043EC      ___exceptStaticBuffP
 0002:000043F0      ___exceptMemAllocVars
 0002:000043F4      ___ExceptStaticXbuff
 0002:00004474      __ExceptVarsSize
 0002:00004488      d62_0
 0002:00004488      __fmode
 0002:0000448C      __fileinfo
 0002:0000448C      d64_0
 0002:00004490      __turboFloat
 0002:00004490      d72_0
 0002:00004494      d78_1
 0002:00004494      __setargv__
 0002:00004498      __argv_expand_ptr
 0002:00004498      d80_0
 0002:0000449C      __wargv_expand_ptr
 0002:0000449C      d82_0
 0002:000044A0      __setenvp__
 0002:000044A0      d86_0
 0002:000044A4      __indStub:44
 0002:000044A8      __indStub:8
 0002:000044AC      __indStub:34
 0002:000044B0      __indStub:6
 0002:000044B4      __indStub:69
 0002:000044B8      __indStub:68
 0002:000044BC      __indStub:70
 0002:000044C0      __indStub:27
 0002:000044C4      __indStub:122
 0002:000044C8      __indStub:7
 0002:000044CC      __indStub:57
 0002:000044D0      __indStub:9
 0002:000044D4      __indStub:55
 0002:000044D8      __indStub:26
 0002:000044DC      __indStub:28
 0002:000044E0      __indStub:25
 0003:00000000      b3_2
 0003:00000020      ___somC_bulletedList_parentMtabs
 0003:00000028      b4_2
 0003:00000028      ___somC_baseType_parentMtabs
 0003:00000038      b5_2
 0003:00000050      ___somC_columnBlock_parentMtabs
 0003:00000068      b6_2
 0003:00000070      ___somC_envProcessor_parentMtabs
 0003:000000AC      b7_2
 0003:000000B4      ___somC_fileMgr_parentMtabs
 0003:000000D4      b8_2
 0003:000000DC      ___somC_footer_parentMtabs
 0003:000000E4      b9_2
 0003:000000EC      ___somC_header_parentMtabs
 0003:000000F4      b10_2
 0003:00000104      ___somC_indentedParagraphs_parentMtabs
 0003:0000010C      b11_2
 0003:0000011C      ___somC_link_parentMtabs
 0003:0000013C      b12_2
 0003:0000014C      ___somC_linkedList_parentMtabs
 0003:00000194      b13_2
 0003:0000019C      ___somC_page_parentMtabs
 0003:000001C4      ___somC_setUpEnvProcessor_parentMtabs
 0003:000001C4      b14_2
 0003:000001D4      b15_2
 0003:000001F4      ___somC_textLine_parentMtabs
 0003:00000208      b16_2
 0003:00000208      ___somC_TPWord_parentMtabs
 0003:00000214      b17_2
 0003:0000024C      ___somC_txtEnvProcessor_parentMtabs
 0003:00000278      b18_2
 0003:00000290      ___somC_word_parentMtabs
 0003:0000124C      b56_2
 0003:0000124C      __DestructorCountPtr
 0003:00001254      ___dll_argc
 0003:00001254      b78_2
 0003:00001258      ___dll_argv
 0004:00000000      ___xxInfo
 0004:00000000      t56_3
